:100000009F018316910107308312990039308316BE
:1000100085003C3087008312071087108510E601A9
:10002000E701E301E401E501831687160716831251
:100030009601161796161615970197171717171684
:10004000971191019115073093009201851D302879
:10005000851D2D288C1A73202828392085103828D2
:100060000313851936288C1A7320312839208514FA
:10007000262887100710051C6228871D5A28071D8F
:1000800044280511051559286508031D49288714BA
:1000900059281F306405433E84000008E9006918B0
:1000A00007141F306405233E84000008E700E40ABB
:1000B000E503612803131610071916146608950046
:1000C00087147228E60CE60C3F30E6058719E61720
:1000D00007196617E71B8714671B0714E70DE70D61
:1000E000FC30E7050034EA01171BEA0A1F306305FC
:1000F000433E84006A0880001F306305233E84006D
:1001000014088000E30AE50A0034FF30EC00FF30F9
:10011000ED008C1E8D2814080800ED0B8928EC0BCF
:100120008728FC348C1E922814080800A000200E9A
:100130000F399E200F3020059E200034A1000A3088
:10014000210203183730031C3030A1072108B120E9
:1001500000342030B12000340D30B1200A30B120FD
:0E0160000034A2008C1CB22822089500003446
:02400E00D230AE
:00000001FF
